:1000000012C0189518951895189518951895189563
:100010001895189518951895189518951895189578
:100020001895189518958FE58DBFC0E4E0E34E2E26
:1000300084E08EBFD4E0F4E05F2EEEEFF3E0A0E6C4
:10004000B0E088278D933197E9F789E189B980E09D
:1000500080BD88E18AB966248EE181BD86E181BDDB
:10006000A098A198A298A398A498A5988A9A8B9AE8
:100070008C9A8D9A8E9A8F9A929893989498959834
:100080009698979880E08093BC0080E08093C100B0
:100090008BE18093BA00AAEBB0E08C91A5EBB0E0C5
:1000A0008D9388278C93A5EBB0E00AD6E8EAF5E1BA
:1000B00041D85CD3E0E0F0E0A2ECB0E056DAE1E059
:1000C000F0E0A3ECB0E051DAE2E0F0E0A4ECB0E064
:1000D0004CDA0091C2000F3F09F00BC00091C30041
:1000E0000F3F09F006C00091C4000F3F09F001C0A6
:1000F00069D5E2E0F0E008D652D538D3DBD20091E2
:10010000C200003009F0DCC081B5886081BDA198D3
:10011000A09890E2A0E6B0E0983018F4392F992723
:1001200002C038E098509999FECF88949899089425
:100130008795999BFECF3A95B1F78D93992361F7F7
:10014000A895EDD1B7D20091C100013009F00CC0E3
:10015000E4EAF5E17BD8EDEBF0E0F1D709D6EDE08C
:10016000F0E0ADEBB0E0D5D90091BC00003009F073
:100170007FC0AAEBB0E08C91C3D5ECEAF5E1B7D52E
:10018000AAEBB0E08C91BCD5E2EBF5E1B0D5E6EBA3
:10019000F5E1ADD5A0EAB0E0A4D5A8E1B4E0A8E1CE
:1001A000B4E0EDEBF0E0552743E038D698D5AAEB64
:1001B000B0E08C91A5D5E0ECF5E199D53CD4AAEB63
:1001C000B0E08C919DD5E4ECF5E191D5AAEBB0E0DF
:1001D0008C9196D5EAECF5E18AD5E6EBF5E187D589
:1001E000A0EAB0E07ED5A8E1B4E0A8E1B4E0EDEB90
:1001F000F0E0552743E012D672D5AAEBB0E08C911F
:100200007FD5E0ECF5E173D516D40091C100013043
:1002100009F015C0AAEBB0E08C9172D5EEECF5E1D7
:1002200066D5E6EDF5E163D5AAEBB0E08C9168D533
:10023000ECEDF5E15CD5E4EEF5E159D518C0AAEB9B
:10024000B0E08C915DD5EEECF5E151D5AAEBB0E0D4
:100250008C9156D5E0ECF5E14AD5AAEBB0E08C9153
:100260004FD5ECEDF5E143D5E4EEF5E140D528C0FE
:10027000AAEBB0E08C9144D5ECEAF5E138D5E6EB99
:10028000F5E135D5A4E6B0E02CD5AAEBB0E08C9131
:1002900037D5AAEBB0E08C9133D5E4ECF5E127D566
:1002A000E6EBF5E124D5A4E6B0E01BD5AAEBB0E07F
:1002B0008C9126D5ECEDF5E11AD5E4EEF5E117D5F4
:1002C0000091C300003009F099C081B5886081BDFC
:1002D000A398A29898E1A0E6B0E0983018F4392FDE
:1002E000992702C038E098509B99FECF88949A993C
:1002F000089487959B9BFECF3A95B1F78D939923F0
:1003000061F7A8950CD1D6D10091BC00003009F05E
:100310004DC0AAEBB0E08C91F3D4E6EEF5E1E7D462
:10032000AAEBB0E08C91ECD4E2EBF5E1E0D4ECEE9A
:10033000F5E1DDD4A0EAB0E0D4D4A8E1B4E0A8E1CE
:10034000B4E0EDEBF0E0552743E068D5C8D4AAEB64
:10035000B0E08C91D5D4E0ECF5E1C9D46CD3AAEB34
:10036000B0E08C91CDD4E6EFF5E1C1D4AAEBB0E0DA
:100370008C91C6D4EAECF5E1BAD4ECEEF5E1B7D451
:10038000A0EAB0E0AED4A8E1B4E0A8E1B4E0EDEBBF
:10039000F0E0552743E042D5A2D4AAEBB0E08C911F
:1003A000AFD4E0ECF5E1A3D446D328C0AAEBB0E08B
:1003B0008C91A6D4E6EEF5E19AD4ECEEF5E197D473
:1003C000A4E6B0E08ED4AAEBB0E08C9199D4AAEB6D
:1003D000B0E08C9195D4E6EFF5E189D4ECEEF5E14F
:1003E00086D4A4E6B0E07DD4AAEBB0E08C9188D4AA
:1003F000ECEDF5E17CD4E4EEF5E179D40091C400B4
:10040000003009F08BC081B5886081BDA598A498A3
:1004100090E2A0E6B0E0983018F4392F992702C096
:1004200038E098509D99FECF88949C9908948795C0
:100430009D9BFECF3A95B1F78D93992361F7A895CF
:100440006ED038D10091BC00003009F03FC0AAEB5B
:10045000B0E08C9155D4ECEFF5E149D4AAEBB0E0D3
:100460008C914ED4E2EBF5E142D4E4E0F6E13FD4E6
:10047000A0EAB0E036D4A8E1B4E0A8E1B4E0EDEB46
:10048000F0E0552743E0CAD42AD4D5D2AAEBB0E095
:100490008C9136D4EEE0F6E12AD4AAEBB0E08C9150
:1004A0002FD4EAECF5E123D4E4E0F6E120D4A0EA8D
:1004B000B0E017D4A8E1B4E0A8E1B4E0EDEBF0E0DF
:1004C000552743E0ABD40BD4B6D228C0AAEBB0E09A
:1004D0008C9116D4E6EEF5E10AD4E4E0F6E107D417
:1004E000A4E6B0E0FED3AAEBB0E08C9109D4AAEB6D
:1004F000B0E08C9105D4E6EFF5E1F9D3E4E0F6E164
:10050000F6D3A4E6B0E0EDD3AAEBB0E08C91F8D33B
:10051000ECEDF5E1ECD3E4EEF5E1E9D3F0CDA4E6C2
:10052000B0E0E0E6F0E0D4D78CE1E4E6F0E004E00F
:100530000A93A5E8B0E0F3D788E1E4E6F0E004E050
:100540000A93AAE8B0E0EBD784E1E4E6F0E004E047
:100550000A93AFE8B0E0E3D780E1E4E6F0E004E03E
:100560000A93A4E9B0E0DBD78CE0E4E6F0E004E035
:100570000A93A9E9B0E0D3D7A5E8B0E0B8D7A4EAD8
:10058000B0E00D931C93AAE8B0E0B1D7A6EAB0E0C2
:100590000D931C93AFE8B0E0AAD7A8EAB0E00D93A2
:1005A0001C93A4E9B0E0A3D7AAEAB0E00D931C9392
:1005B000A9E9B0E09CD7ACEAB0E00D931C9387E0CA
:1005C000E4E6F0E001E00A93AEE9B0E0A8D7AEE9D6
:1005D000B0E0E6E1F6E1D3D709F006C0A0EAB0E06A
:1005E000E8E1F6E1A7D505C0A0EAB0E0EAE1F6E16E
:1005F000A1D585E0E4E6F0E001E00A93A2EAB0E0EC
:100600008ED7A2EAB0E0ECE1F6E1B9D709F02CC050
:10061000AEEAB0E0ECEAF0E006D7AEEAB0E050D3E4
:10062000EAEAF0E000D7AEEAB0E04AD3E8EAF0E068
:10063000FAD6AEEAB0E044D3EEE1F6E17BD5AEEA1D
:10064000B0E03ED3E6EAF0E0EED6AEEAB0E038D372
:10065000E4EAF0E0E8D6AEEAB0E001D6EDE0F0E0A2
:10066000ADEBB0E056D725C0AEEAB0E0EAEAF0E084
:10067000DAD6AEEAB0E024D3EEE1F6E15BD5AEEA3D
:10068000B0E01ED3E8EAF0E0CED6AEEAB0E018D390
:10069000E6EAF0E0C8D6AEEAB0E012D3E4EAF0E071
:1006A000C2D6AEEAB0E0DBD5EDE0F0E0ADEBB0E015
:1006B00030D708950CD3ABEBB0E08C930091BB0026
:1006C000003010F009F001C03FC082E6482F0091D1
:1006D000BB00041709F003C081E08093BC0083E6EF
:1006E000482F0091BB00041709F001C0F2D184E645
:1006F000482F0091BB00041709F006C080E08093EA
:10070000BC0080E08093C10085E6482F0091BB00CB
:10071000041709F001C056D286E6482F0091BB00AD
:10072000041709F001C0AAD182E7482F0091BB004D
:10073000041709F003C081E08093C1000091BB0061
:100740000B3109F001C012D0AAEBB0E08C91D8D2E5
:10075000ECEDF5E1CCD2E4EEF5E1C9D2AAEBB0E0E4
:100760008C91CED2E0ECF5E1C2D20895A5EBB0E0D9
:10077000B8D2AAEBB0E08C91C3D2E0E2F6E1B7D2F6
:10078000AAEBB0E08C91BCD2E6E2F6E1B0D2A5EBE8
:10079000B0E0A7D2AAEBB0E08C91B2D2ECE2F6E1E5
:1007A000A6D2E4E3F6E1A3D2A8D2AAEBB0E08C9102
:1007B000A7D2E6E5F6E19BD2EEE5F6E198D29DD22E
:1007C000AAEBB0E08C919CD2ECEAF5E190D2AAEBD6
:1007D000B0E08C9195D2E2EBF5E189D2E6EBF5E160
:1007E00086D2AAEBB0E08C918BD2E4ECF5E17FD21B
:1007F000AAEBB0E08C9184D2EAECF5E178D2E6EB9A
:10080000F5E175D2AAEBB0E08C917AD2E6EEF5E193
:100810006ED2AAEBB0E08C9173D2E2EBF5E167D235
:10082000ECEEF5E164D2AAEBB0E08C9169D2E6EF90
:10083000F5E15DD2AAEBB0E08C9162D2EAECF5E191
:1008400056D2ECEEF5E153D2AAEBB0E08C9158D23F
:10085000ECEFF5E14CD2AAEBB0E08C9151D2E2EB97
:10086000F5E145D2E4E0F6E142D2AAEBB0E08C91AA
:1008700047D2EEE0F6E13BD2AAEBB0E08C9140D259
:10088000EAECF5E134D2E4E0F6E131D2AAEBB0E0F3
:100890008C9136D2E6E7F6E12AD2EEE7F6E127D2EE
:1008A000AAEBB0E08C912CD2E0EAF6E120D2E8EAA3
:1008B000F6E11DD2AAEBB0E08C9122D2EAECF6E18F
:1008C00016D2E2EDF6E113D2AAEBB0E08C9118D289
:1008D000E4EFF6E10CD2ECEFF6E109D2AAEBB0E0DE
:1008E0008C910ED2EEE1F7E102D2E6E2F7E1FFD120
:1008F000AAEBB0E08C9104D2E8E4F7E1F8D1E0E5AE
:10090000F7E1F5D1AAEBB0E08C91FAD1E2E7F7E19B
:10091000EED1EAE7F7E1EBD1AAEBB0E08C91F0D1B0
:10092000ECE9F7E1E4D1E4EAF7E1E1D1AAEBB0E0E8
:100930008C91E6D1E6ECF7E1DAD1EEECF7E1D7D134
:10094000AAEBB0E08C91DCD1ECEDF5E1D0D1E4EE96
:10095000F5E1CDD1AAEBB0E08C91D2D1E0ECF5E19C
:10096000C6D10091C2000F3F09F01EC0AAEBB0E053
:100970008C91C6D1ECEAF5E1BAD1E0EFF7E1B7D15D
:10098000AAEBB0E08C91BCD1E4ECF5E1B0D1E0EFA2
:10099000F7E1ADD1AAEBB0E08C91B2D1ECEDF5E18D
:1009A000A6D1E4EEF5E1A3D10091C3000F3F09F019
:1009B0001EC0AAEBB0E08C91A3D1E6EEF5E197D191
:1009C000E0E0F8E194D1AAEBB0E08C9199D1E6EFA8
:1009D000F5E18DD1E0E0F8E18AD1AAEBB0E08C91AD
:1009E0008FD1ECEDF5E183D1E4EEF5E180D100911A
:1009F000C4000F3F09F01EC0AAEBB0E08C9180D17B
:100A0000ECEFF5E174D1E0E1F8E171D1AAEBB0E0EF
:100A10008C9176D1EEE0F6E16AD1E0E1F8E167D1C0
:100A2000AAEBB0E08C916CD1ECEDF5E160D1E4EE95
:100A3000F5E15DD10895A2EAB0E0ECE1F6E19FD5E1
:100A400009F00EC0E0E2F8E152D1AAEBB0E08C91DF
:100A500057D1ECEDF5E14BD1E4EEF5E148D10DC015
:100A6000E6E2F8E144D1AAEBB0E08C9149D1ECED9B
:100A7000F5E13DD1E4EEF5E13AD10895929A88E2AC
:100A800090E051D1929888EC90E04DD1939A88E211
:100A900090E049D19398A895959A88E290E043D147
:100AA000959888EC90E03FD1949A88E290E03BD111
:100AB0009498A895979A88E290E035D1979888EC19
:100AC00090E031D1969A88E290E02DD19698A89541
:100AD0000895AAEBB0E08C9113D1ECEDF5E107D1CC
:100AE000ECE2F8E104D1AAEBB0E08C9109D1E0ECA2
:100AF000F5E1FDD0ECD0ABEBB0E08C93A895009184
:100B0000BB00003010F009F001C02FC08AE7482F69
:100B10000091BB00041709F006C0939A8CE291E0A3
:100B200002D19398A89589E7482F0091BB0004173C
:100B300009F006C0949A8CE291E0F5D09498A895BB
:100B400088E7482F0091BB00041709F006C0969A69
:100B50008CE291E0E8D09698A89581E6482F009124
:100B6000BB00041709F001C01AD00091BB0000308F
:100B700010F009F001C0BECFAAEBB0E08C91C0D05C
:100B8000ECEDF5E1B4D0E4EEF5E1B1D0AAEBB0E0E4
:100B90008C91B6D0E0ECF5E1AAD0A8950895939A8F
:100BA0008CE291E0C0D09398A895949A8CE291E061
:100BB000BAD09498A895969A8CE291E0B4D0969881
:100BC000A8950895AAEBB0E08C919AD0ECEDF5E1F0
:100BD0008ED0E4EEF5E18BD0AAEBB0E08C9190D012
:100BE000E0ECF5E184D0E0E5F8E181D070D0ABEB4A
:100BF000B0E08C930091BB00003010F009F001C010
:100C000055C088E7482F0091BB00041709F00BC0BE
:100C100080E08093C200E0E0F0E0A0E1BB2780E04C
:100C20008C937BE791D489E7482F0091BB00041790
:100C300009F00BC080E08093C300E1E0F0E0A0E1A8
:100C4000BB2780E08C937BE77FD48AE7482F009115
:100C5000BB00041709F00BC080E08093C400E2E001
:100C6000F0E0A0E1BB2780E08C937BE76DD48CE6BD
:100C7000482F0091BB00041709F018C0E0E0F0E035
:100C8000A0E1BB278FEF8C937BE75ED4E1E0F0E03F
:100C9000A0E1BB278FEF8C937BE756D4E2E0F0E036
:100CA000A0E1BB278FEF8C937BE74ED4A8950091F2
:100CB000BB000D3009F09ACF59DD0895F894FFCFAD
:100CC0008F938D918823E9F711978F910895882745
:100CD0005F9B089500C05F9BFECF8CB10895A8E193
:100CE000B4E08D91882311F00BD0FBCF0895AAD2E8
:100CF000802D11F005D0FBCF08958DE001D08AE062
:100D00005D9BFECF8CB9089588EE93E00CD03197AF
:100D1000D9F708953197F1F70895689462F8089526
:100D2000E89462F80895EF93FF93EE27E82BE92B00
:100D300031F0E0EAFFE03197F1F70197D1F7FF9149
:100D4000EF9108958F939F93D216E306F4060FB6A2
:100D500080E890E8802795270FBE89070FB6892B7A
:100D600087FD02C091E009260FBE9F918F910895E3
:100D700043D0A9F0503899F01627050F1BF40AF05C
:100D800038C23EC203951BD0FF202AF0BB0CDD1CED
:100D9000EE1CFF1C02C003951BF003D0DAC130C269
:100DA00028C2B7FE089590E8B91611F4D0FE089550
:100DB0009FEFD91AE90AF90A09F403950895FF92F9
:100DC000EF928D2DFF24EE24DD24BB2493E0849F3D
:100DD0001001829FB00CD11CE21CF31C839FD00C2D
:100DE000E11C2224F21C9A9531F0BD2CDE2CEF2C54
:100DF000FF248F91ECCF0895652F90E8440F551F85
:100E00005927990F47956078102F90E8FF0C001F25
:100E10000927990FF79410780038089590D1F4DFDE
:100E200017FF03C08DE28D931127003819F4E8ED08
:100E3000F0E180C10F3741F4FF2019F4EEECF0E14E
:100E4000F8CFEAECF0E1F5CF4A934A934A935A93EC
:100E5000BA93AA93BB270F5FCAF4BB27802F0A95CA
:100E600078D18D3E70F4E8E2F1E1A3E0EFD16ADFE2
:100E7000BB1FB0FF04C07097E9D17ADF3C96AA95FA
:100E8000A9F7E4E2F1E1E2D173DF1DC0093028F1F6
:100E9000033148F10A3130F418E08BE192E9ECEDCE
:100EA000F0E128C00A9555D1ECE1F1E1BFEFA3E0F4
:100EB000CDD148DFBB1FB0FD04C03896C7D158DF85
:100EC0003C97AA95A9F7B095BB0F9EDF039513E059
:100ED0008AEF99E0F816090740F413E08BE094E0FC
:100EE000E0EFF0E107C016E001C0B39583E194E2C2
:100EF000E4EEF0E16A81BF3F19F4BB27112762607D
:100F0000BD836A831C83A881B98160E36D93A88344
:100F1000B9836D93081B0195AA24BB246A816A7F5B
:100F2000002339F0F694E794D794B794A7940A95E0
:100F3000F7CF19E000278AD1CC248FEF74E0AC14EE
:100F4000B206D306E406F50630F0AC18B20AD30AAE
:100F5000E40AF50A21F1881F7A9531F056954795F4
:100F600037952795C794EBCF809522D041F0969581
:100F700010F7FE2CED2CDB2CBA2CAA24DCCF25D0CC
:100F80005D813C812B8170D0277021F02BD06CD0FB
:100F9000E8F301C03CD04CD078D0269608958894D0
:100FA000881F7A95E9F7809503D049F38827FCCF0D
:100FB000806360FD06C0803311F0616002C003955C
:100FC00061FD8D9360FD1A95089599278E919C93EC
:100FD00085338E9108F083958A3308F080E38C93F3
:100FE000C0F70895732F720F61FF701B0AD012961D
:100FF000785019F050F38E9380E38E937150EAF796
:101000000895A881B981A70F8827B81F089579E0AE
:1010100061FD700FF6DF48E0431B400F8AF381F358
:1010200099274A9569F38E91803351F79C93F9CFB4
:10103000732F61FF701B7395A881B981EA2FFB2F75
:1010400011978191803361FF09F08D937A9511F4A6
:101050008EE28D9381918823C1F7772311F480E389
:101060008D9388278C930895889462FD08950023BA
:1010700059F4A881B9818C91803331F0552321F046
:10108000539533506460089408955523E9F085E43E
:101090008D931AF48DE28D935195652F660F560F3F
:1010A0005A3010F060E503D068E001D0DACF8FEF5E
:1010B00074E0561708F0561B881F7A9511F0669554
:1010C000F8CF809580638D9308954E414E00496E10
:1010D00066696E6974790000302E300000404B4C18
:1010E0000020A107000050C3000088130000F40195
:1010F000000000320000000500008000CCCCCC0CC9
:1011000014AE47019CC42000DC460300E3530000FA
:1011100063080000D7000000150000001CC25367E0
:10112000A5D468530024744915BE9A17CCBC8C2BE7
:10113000BD37863587D00D920020E1F70895D19014
:10114000E190F19001910895219131914191519156
:101150000895FF0C90E89027110F9795F794092FA9
:101160000895502F2D2D3E2D4F2D612F08952DECDC
:101170003CEC4CEC5DE366270FC0E1DFF2DFDD24E1
:10118000EE2490E8F92E0FE307C0DEDF05C022272A
:10119000332740E251E46627552351F1002381F1C2
:1011A0002BDE71F11627005850580894050B18F4DF
:1011B00007FD03C025C007FD23C046953795279539
:1011C000F694E794D79422D0FF202AF0DD0CEE1C91
:1011D000FF1C015073F09D2D969548F0DD203AF4E8
:1011E000EE202AF491E0D90E9927E91EF91EB1CF1D
:1011F00007C09FE7092FF92A9FEFD92EE92E0895FE
:10120000DD24EE24FF240027112708959F929924BE
:10121000AA24BB2488E1D216E306F40628F0D21AE9
:10122000E30AF40A089401C08894991CAA1CBB1C08
:10123000DD0CEE1CFF1C8A9571F7D92CEA2CFB2CD7
:101240009F900895C895319600200895FBDF202DCA
:10125000F9DF302DF7DF402DF5DF502D089560DDEB
:10126000E89488278A938A93CBDF11278D91803267
:10127000E9F31197BAD090F08D3229F410951196B8
:101280008C91B3D058F08E3229F411968C91ADD058
:1012900008F445C0229641DD81E008958C91A5D0E7
:1012A000D8F547D01196D0F703958D919ED0E0F3F5
:1012B0008E3229F48C9199D010F41196FBCF85349D
:1012C00019F0853609F055C011968C918ED060F0DA
:1012D0008D3219F08B3221F0DDCF08800094088226
:1012E00011968C9182D0B0F68053898311968C919F
:1012F0007CD058F49981990F990F0980900D990F1E
:101300008053890F8983873228F6898198819923B0
:101310000AF48195080F2DC08E3289F611968C91B2
:1013200064D068F606D018F011960A95F8CF119699
:10133000C1CF4F2D3E2D2D2DDD0CEE1CFF1CA8F036
:10134000DD0CEE1CFF1C88F0D20EE31EF41E68F0CC
:10135000DD0CEE1CFF1C48F0805309F06894D80E99
:101360008827E81EF81E08F00895F42EE32ED22EEA
:10137000089534D019F116F5098308E921D00695AE
:10138000882787959F2D9F77980FF92E0150000F82
:10139000110F07958981882379F01AF48195898343
:1013A00006C0E5DE89818A958983D9F705C0EFDE1D
:1013B00089818A958983D9F72296089521DFFCCF08
:1013C0000DD041F0FF2032F00A9531F0DD0CEE1C1B
:1013D000FF1CD2F7889408950894089500240D28DE
:1013E0000E280F28002A00200895803320F08A3329
:1013F00010F40894089588940895000F111F221F77
:10140000331F089500951095209530950F5F1F4F5D
:101410002F4F3F4F0895019110810EC001911191FE
:10142000219130810BC00191108117FF05C03FEF62
:101430002FEF04C0008111272227332737FF03C075
:10144000E1DF8DE28D93CF93DF93CF92DF92EF9226
:10145000AA24BB24CC24DD24EE2440E2CAE0DD270C
:1014600055E093E38881890F87FD9F7083FD907F0E
:10147000891B89935A95A9F7C0DFAA1CBB1CCC1CF9
:10148000DD1CEE1C4A9551F7E894EFE0FF278291AE
:101490000ED0EB30E0F71EF068948A2D0CD0882730
:1014A0008D93EF90DF90CF90DF91CF910895982F9B
:1014B000829501D0892F8F70805D26F0803309F4EA
:1014C000089568948D93089541E003C042E001C0FF
:1014D00044E0E40F8827F81F829138E098E1880FF4
:1014E000991F9D933A95D1F74A95B1F70FC0002700
:1014F0001127222733278D91882339F08053000F3D
:10150000111F221F331F080FF6CF089588278D93D0
:10151000089594E081918D939A95E1F7089509914A
:101520009191992351F08A95D9F7319781918D93B3
:101530000A9519F08823D1F70895E8CFE199FECFF5
:10154000EEBBFFBB3196089591E001C092E07B377E
:1015500051F47FB7F894F2DF8D918DBBE29AE19A56
:101560009A95C9F77FBF7727089591E001C092E06F
:10157000E5DFE09A8DB38D939A95D1F7089568943D
:1015800001C0E894AF93BF938D9116F0919102C082
:1015900059DE902D891718F011F48823A9F7BF910F
:1015A000AF910895000000405B324A005B353B314B
:1015B000480023330000582D4163687365203A00CA
:1015C0005B4B00005B363B314800233400005B324C
:1015D000323B33364800616B746976005B31343BD3
:1015E000314800003E005B383B314800592D4163D3
:1015F000687365203A005B393B3148005B31313B11
:10160000314800005A2D4163687365203A005B3110
:10161000323B3148000030002B002D0031002E00FD
:101620005B34316D00005B33376D00005B313B3262
:10163000304800004D657373736368696562657255
:10164000204175736C6573652053797374656D20E3
:1016500056312E3100005B323B3235480000A92064
:1016600048616E7320426F726E6772616562657267
:101670002032303038005B31363B32480000C9CD73
:10168000CDCDCDCDCDCDCDCDCDCDCDCDCDCDCDCD8A
:10169000CDCDCDCDCDCDCDCDCDCDCDCDCDCDBB0059
:1016A0005B31373B32480000BA20622020203D20C9
:1016B00062696E6165722020202020202020202079
:1016C0002020202020202020BA005B31383B3248E7
:1016D0000000BA20632020203D20636C65617220E9
:1016E00020202020202020202020202020202020FA
:1016F0002020BA005B31393B32480000BA20642018
:1017000020203D2064657A696D616C2020202020B6
:10171000202020202020202020202020BA005B3202
:10172000303B32480000BA20652020203D2065690A
:101730006E7269636874656E20202020202020204E
:10174000202020202020BA005B32313B32480000AC
:10175000BA20662020203D20666173742072656186
:10176000642065696E2F6175732020202020202061
:10177000BA005B32323B32480000BA20722020208F
:101780003D2044757263686D65737365722F526195
:1017900064697573202020202020BA005B32333B1F
:1017A00032480000BA20455343203D2042696C6412
:1017B00073636869726D206E65752061756662611C
:1017C00075656E20BA005B32343B32480000C8CDEC
:1017D000CDCDCDCDCDCDCDCDCDCDCDCDCDCDCDCD39
:1017E000CDCDCDCDCDCDCDCDCDCDCDCDCDCDBC0007
:1017F000582D4163687365203A206E2E612E0000DB
:10180000592D4163687365203A206E2E612E0000C9
:101810005A2D4163687365203A206E2E612E0000B8
:10182000206D6D20200020696E6368003E57656C56
:1018300063686520416368736520617566204E7535
:101840006C6C2028782C792C7A2C61293F200000A0
:1018500057656C6368652041636873656E207369C2
:101860006E6420616E67657363686C6F7373656E19
:0A187000202878797A2C6C293F00BB
:00000001FF
